:100648001C2C2863292032303030205345474D4533
:100658004E542062762C2076312E312E3700024EF1
:100668000000C187C182C189C184C106C100C10817
:10067800C103C10BC10AC1010122000250000001DF
:100688004D000156000A57CDA348C285CD91CFA38E
:10069800C80452C7CF48910923FDFEFBF7EFDFBF1F
:0706A8007FFF034A01010777
:10000D00D2B0D2B1758903D28CD2AFD2A97F807E06
:10001D003ED136300007300804B1AE80F0E4F51261
:10002D007F5C7E44D13674522512F8E6F5907F5CE4
:10003D007E44D1367590FF0512C3E5126480948419
:10004D0040DED2B7AF4DD20C719A300A0221273063
:10005D00003F30B721D3E54D6480948E5009C3E540
:10006D004D648094815005754D018002054DAF4D55
:10007D00D20C719A8019E522D39412400575220194
:10008D0080020522AF22C20C719AE4F54EF54FC2E3
:10009D000030083630B718C3E54D648094825005A2
:1000AD00754D0F8002154DAF4DD20C719A8019E52B
:1000BD0022C39402500575221380021522AF22C26D
:1000CD000C719AE4F54EF54FC20830061CA2B7B379
:1000DD009205A20592B7200508AF22C20C719A8035
:1000ED0006AF4DD20C719AC20630032EE54D700A43
:1000FD00D2B77F15C20C719A801EE522700AC2B765
:10010D007F16C20C719A8010E4F563F564F5508585
:10011D002251D20AF510F511C203200A020157919E
:10012D008CE556FD3395E0FCAE4EAF4FF172ED4CC4
:10013D006006ED64014C7004D20B8002C20B2000EE
:10014D000330080A75109C751140C200C2083006B4
:10015D000AB2B775109C751140C206200304E52242
:10016D007025C20BC206C200C208C203C20AE52234
:10017D007002F54D20B708AF22C20C719A0157AF2E
:10018D004DD20C719A0157D3E5119420E510944E80
:10019D00401DC20120B708AF22C20C719A8006AF74
:1001AD004DD20C719AE5111511700215100157D22F
:0401BD0001015722C3
:02000B0021C111
:1001C100C0E0C0F0C0D075D0080564E564700205D8
:1001D10063300A2AD3E56494A2E56364809487407E
:1001E1001DE4F563F564054FE54F7002054EAE4E13
:1001F100AF4F7C007D78F172ED4C70021522200129
:1002010002418BD296D297C3E56494F4E56364808E
:10021100948050057590FD806FC3E56494E8E563B3
:100221006480948150057590FE805DC3E56494DC23
:10023100E5636480948250057590BF804BC3E5648B
:1002410094D0E5636480948350057590EF8039C341
:10025100E56494C4E5636480948450057590F780E7
:1002610027C3E56494B8E56364809485500575906F
:10027100FB8015C3E56494ACE56364809486500506
:100281007590BF80037590DFC201A2B5300701B33D
:100291004018A2B3300201B34010A2B4300901B337
:1002A1004008A2B2300401B35015A2B59207A2B31F
:1002B1009202A2B49209A2B29204E4F548F549A2CD
:1002C100B5300701B3406EA2B3300201B34066A25C
:1002D100B4300901B3405EA2B2300401B340560507
:1002E10049E54970020548E549642845487016A268
:1002F10007B39206A202B39200A209B39208A20424
:10030100B392038030E549B49411E548B4110CA2CD
:1003110002B39200A209B39208801AE549B4EC1520
:10032100E548B41310A202B39200A209B392087572
:100331004811754994E56245617013300B0A0562F5
:10034100E56270020561804AD2B0D2B18044056293
:10035100E56270020561E562640245617004D2B034
:100361008030E562640345617004C2B08024E562B7
:10037100641445617004D2B18018E5626415456169
:100381007004C2B1800CE562642545617004F561B9
:09039100F562D0D0D0F0D0E032CA
:10039A00EFB417004002818B9003A825E07361D661
:1003AA0061E161E561E961ED61F161F561F961FDC3
:1003BA00810181058110811B81268131813C814720
:1003CA00814B814F8153818B81578171200C047538
:1003DA0090C0227590F7227590FA227590A4227522
:1003EA0090B02275909A227590912275908122750B
:1003FA0090F8227590802275909022200C047590B6
:10040A00402275908822200C0475907A2275908378
:10041A0022200C04759024227590C522200C0475A4
:10042A009030227590A222200C0475901A227590A1
:10043A008522200C047590112275908D22759001E9
:10044A002275907822E4F5902275901022200031CE
:10045A0020082E7590FF7F707E17D1367590F77F32
:10046A00887E13D13680E62000172008147590FF85
:10047A007F707E17D1367590C07F887E13D1368003
:02048A00E62268
:10048C00E54D75F002F13CAFF0EF7008790A7B078F
:10049C007A05800679097B067A03C3E54D6480945E
:1004AC008A5008C3740C954DF55622C3E54D6480F3
:1004BC00948C505BAE50AF517C007D18F15EC3E55F
:1004CC004F9FE54E9E5003895622AE50AF517C0093
:1004DC007D24F15EC3E54F9FE54E9E50038B562263
:1004EC00AE50AF517C007D60F15EC3E54F9FE54E91
:1004FC009E50038A5622AE50AF517C007D6CF15E4B
:10050C00C3E54F9FE54E9E50038B5622895622C35E
:10051C00E54D6480948E502FAE50AF517C007D24FD
:10052C00F15EC3E54F9FE54E9E5003895622AE50B7
:10053C00AF517C007D48F15EC3E54F9FE54E9E5068
:10054C00038B56228A5622AE50AF517C007D18F197
:10055C005EC3E54F9FE54E9E50038B5622AE50AFC7
:10056C00517C007D30F15EC3E54F9FE54E9E5003FC
:10057C008A5622AE50AF517C007D48F15EC3E54FE8
:10058C009FE54E9E50038B5622AE50AF517C007DA2
:10059C0060F15EC3E54F9FE54E9E50038A56228B59
:0205AC005622D5
:1005AE00E4F5137590FFC206C203300322E4F5137F
:1005BE007F207E4ED13674232513F8E6F590B2B720
:1005CE000513C3E5136480948940E5B2B7C20330C6
:1005DE0006D8E4F5137F207E4ED13674572513F8D6
:1005EE00E6F5907F207E4ED1367590FF0513C3E55C
:1005FE00136480948A40DEE4F5137F207E4ED1365C
:10060E00744A2513F8E6FFC20C719A7F207E4ED1F4
:10061E00367590FF0513C3E5136480948340DBC2E7
:08062E0006C200C208C203224B
:10063600E4FDFCC3ED9FEC9E50070DBD00010C8050
:02064600F2229E
:030000000206B045
:0C06B000787FE4F6D8FD7581640206F73F
:10073C00C2D530F707B2D563F0FF05F030E70CB245
:10074C00D5F4048463F0FF05F080018430D502F405
:02075C00042275
:10075E00EFF88DF0A4FFEDC5F0CEA42EFEEC88F0E0
:04076E00A42EFE2295
:10077200C2D5EC30E709B2D5E4C39DFDE49CFCEEA2
:1007820030E715B2D5E4C39FFFE49EFE1207A8C36B
:10079200E49DFDE49CFC80031207A830D507C3E466
:0607A2009FFFE49EFE2211
:1006BC0002000DE493A3F8E493A34003F68001F247
:1006CC0008DFF48029E493A3F85407240CC8C3333F
:1006DC00C4540F4420C8834004F456800146F6DF0E
:1006EC00E4800B0102040810204080900648E47E50
:1006FC00019360BCA3FF543F30E509541FFEE49303
:10070C00A360010ECF54C025E060A840B8E493A3C9
:10071C00FAE493A3F8E493A3C8C582C8CAC583CAF4
:10072C00F0A3C8C582C8CAC583CADFE9DEE780BEAC
:0106AF00004A
:1007A800BC000BBE0029EF8DF084FFADF022E4CC35
:1007B800F875F008EF2FFFEE33FEEC33FCEE9DECFE
:1007C800984005FCEE9DFE0FD5F0E9E4CEFD22ED44
:1007D800F8F5F0EE8420D21CFEADF075F008EF2F8E
:1007E800FFED33FD4007985006D5F0F222C398FD7F
:0507F8000FD5F0EA221C
:00000001FF
